:020000040000FA
:0400000000002628AE
:08000800A00003088301A10020
:100010000A08A2000408A30083160C08403903193B
:100020001C2883120C088316403903191C288312DC
:100030001E08A6000C139F148301230884002208C5
:100040008A0021088300A00E200E0900FF238316DA
:100050009000D830850083128501831699018312A0
:100060000730990083160C1783120B170C138B178C
:10007000831618309F0083120D309F00000000008F
:10008000000000009F140330A500A60125080339D5
:1000900082074D2853285E285E28AD3026020318BB
:1000A0005228A50A6328B2302602031C5828A5034B
:1000B0004230260203185D28A50A63284C30260228
:1000C000031C6328A5032508033982076A286E28C4
:1000D0007228722883123B308500462883123D30F7
:0C00E0008500462883121F30850046284A
:1006600045344C3445344334543452344F344E348E
:100670004934433420344C344534563445344C34B6
:1006800045345234203450344934433420343134E6
:1006900032344634363437343534203442345934E5
:1006A000203444345234203452342E3420344534EF
:1006B00052344C34493443344834203463342F3476
:1006C0006F342034453449344434203443344F3477
:1006D000523450342E34203441344E344434203497
:1006E0004234593420344B3445344934543448343A
:1006F000203459344F3455344E34473442344C341A
:100700004F344F344434203463342F346F34203426
:1007100059344234203454344534433448342E342C
:1007200020344134553447342E342034323430347C
:1007300030343834203420342034203420342034F1
:100740002034203420342034203420342034203409
:1007500020342034203420342034203420342034F9
:100760005434483449345334203453344F344634A9
:10077000543457344134523445342034493453349A
:100780002034503452344F34563449344434453490
:10079000443420344F344E34203441344E342034E9
:1007A00041345334203449345334203443344F34A7
:1007B0004E3444344934543449344F344E342E3456
:1007C0002034203420342034203420342034203489
:1007D0002034203420342034203420342034203479
:02400E00843FED
:00000001FF
